:0200000480007A
:100000006F008004732F2034930F80006308FF0378
:10001000930F90006304FF03930FB0006300FF038E
:10002000130F000063040F0067000F00732F2034CC
:1000300063540F006F00400093E19153171F0000BD
:1000400023223FFC6FF09FFF732540F163100500F2
:10005000970200009382020173905230735000188F
:10006000970200009382020273905230B702008020
:100070009382F2FF7390023B9302F0017390023A75
:1000800097020000938282017390523073502030A7
:1000900073503030735040309301000097020000DD
:1000A000938282F673905230130510001315F501F8
:1000B000634C05000F00F00F930110009308D0056A
:1000C00013050000730000009702000093820209EC
:1000D000638E020073905210B7B2000093829210A8
:1000E0007390223073232030E39862F47350003011
:1000F0003715000013050580732005301305200215
:1001000073203530970200009382420173901234BD
:10011000732540F17300203093012000730010001C
:100120006F008000631030020F00F00F6380010049
:100130009391110093E111009308D00513850100FC
:10014000730000000F00F00F930110009308D0051A
:10015000130500007300000013033000F322201485
:10016000E39462FC17030000130383FBF3221014D3
:10017000E39C62FA6FF01FFD731000C000000000E6
:1010000000000000000000000000000000000000E0
:1010100000000000000000000000000000000000D0
:1010200000000000000000000000000000000000C0
:1010300000000000000000000000000000000000B0
:081040000000000000000000A8
:040000058000000077
:00000001FF
